:1000000000308A00B22900000A108A100A11820703
:1000100028340C34013406340A108A100A1182077D
:100020000C34413468346F346A34213400340A109B
:100030008A100A11820776347934733469346C3447
:1000400061346D3400342E308400000803193728E1
:100050000130A100A001A00B2B28A10B2A284A30B7
:10006000A000A00B312800000000800B28280034DD
:1000700006080F39B500340EA000F030A0052008A6
:10008000F039350486000615831606110000831228
:1000900006118316061183120034B208031D52287C
:1000A000861053288614831686108312B30E3308E5
:1000B000B4003820B30E3308B40038200D30A0004F
:1000C000A00B602800341430AE0023200F308316BC
:1000D00086058312861083168610831206118316F6
:1000E00006118312AB012B08023C031C7F2802304F
:1000F000AE0023200330B4003820AB0A73280D3043
:10010000A000A00B81280230B40038200D30A000E0
:10011000A00B8828AB012B08023C031C9B282B0852
:100120000420AC00B2012C08B3004D200230AE0018
:100130002320AB0A8B288A11F42901302E02B0004B
:100140002F08023C031DA6284030B0073008803835
:10015000B100B2013108B3004D2000342D08A000D9
:100160000C3020020319C1280A3020020319C928C3
:100170000D3020020319CF28083020020319D4289B
:10018000D928B2010130B3004D200230AE00232047
:10019000E5280130AE000230AF009D20E528013097
:1001A000AE00AF009D20E528B2011030B3004D2015
:1001B000E5282D081F3C031CDF280730AD05013062
:1001C000B2002D08B3004D20E52800342E08A1010F
:1001D0002D020318EE282D08A000FA28A0010830EF
:1001E000AF00AD0DA00D2E0820020318A000A10D38
:1001F000AF0BF12800342B08A000AB1B03292C1DEA
:100200000D2920300829A009A00A2008AB002D30B4
:10021000A100AD00AE202C1DAC152B08AD00643044
:10022000AE00E6202008AB0021083030031D1F2956
:100230002C18AC15AC1925292C1A20302129AC1109
:100240002C12A1072108AD00AE202B08AD000A300A
:10025000AE00E6202008AB0021083030031D342911
:10026000AC1938292C1A2030A1072108AD00AE2086
:100270003030AB072B08AD00AE200034AF012F08A3
:10028000073C031C96292E08A0002F08A100031983
:100290004D290310A00CA10B492900302018013072
:1002A000013C031D6B29A9112908831687008312BD
:1002B0008715A630A000A00B5B290000A911290812
:1002C0008316870083128711F930A000A00B6629DE
:1002D000000000009429A9112908831687008312C1
:1002E00087155330A000A00B7329A9112908831684
:1002F000870083128711A630A000A00B7D29000083
:10030000A911290883168700831287155330A0008E
:10031000A00B8829A9112908831687008312871149
:100320005330A000A00B9229AF0A3F2900340F30B0
:10033000AB002B08AE003E218A11902A2B0EA000A4
:10034000F030A00520082B07AD00AE003E212C0E9A
:10035000A000F030A00520082C07AD00AE003E2123
:100360008A11952A84011F308305073083169F0068
:10037000FF308312A900AA01043083169F00831264
:100380001F08383901389F009412A91229088316D2
:100390008700831229162908831687008312A91162
:1003A0002908831687000030831294008316940076
:1003B0008312A001A01DE42907308101813084004F
:1003C0000008C0390F3880006400813084000008C4
:1003D000C0392004800090010030A100920000305C
:1003E00083169200831263282A08103C031C082AF3
:1003F0002A08AE000130AF009D205F30AD00AE2076
:100400003230AE0023200C30AD00AE20AA0AF42911
:10041000AB012B080C20AB0AAD00AE2006302B023E
:10042000031D092A0630AB00FA30AE002320AB0BC7
:10043000142A0C30AD00AE200030A1001F08C739CF
:1004400021049F000130AE00AF009D201F151F1931
:10045000272A1E081E0EA7000F30A7055830AD0032
:10046000AE203A30AD00AE202030AD00AE202708DF
:10047000AB001830AC00FB200630AB002030AD00E4
:10048000AE20AB0B3E2A0830A1001F08C73921045B
:100490009F000130AE000230AF009D201F151F19D4
:1004A0004F2A1E081E0EA8000F30A8055930AD00B7
:1004B000AE203A30AD00AE202030AD00AE2028088E
:1004C000AB001830AC00FB200630AB002030AD0094
:1004D000AE20AB0B662A0730AE000230AF009D2085
:1004E000AB012B081720AB0AAD00AE2007302B0262
:1004F000031D712A29122908831687008312071603
:100500002913290883168700831207170130AE00CC
:10051000232029122908831687008312071297299E
:100520002708AB002808AC009E2929132908831648
:0A0530008700831207131C2A6300E2
:02400E00F13F80
:00000001FF
